:020000001B29BA
:1000060002308312FC004930FD00FD0B0828FC0B72
:080016000828000000000800AA
:0E001E000E308312FD00FD0B122800000800BA
:0C002C00831228088A00270882000800C0
:10003800FF308312A400FF30A500FF30A600FF3078
:10004800C3309F05F0309F05F03083169F0483125C
:060058009F171F140800B1
:10005E00C33083129F05F0309F05F03083169F0446
:10006E0083129F172D08F000F00D7010F00D701018
:10007E0070089F041F140F209F149F1C4828000017
:10008E0044281F101E08F100F00183161E08F0040C
:06009E000030F10408002F
:1000A4000930831685008B01831290010730990073
:1000B40083169901813083129F00513083169F006B
:0600C40083128501080013
:1000CA008312B2012E08F1000130F0007108031901
:1000DA007228F00D7010FF3E6C287008B1002D08D0
:1000EA00840070080005F10071080130031D00301A
:1000FA00F0003008F00603199A282F08003C03186C
:10010A008A2803200320AF0382282D08840031089F
:10011A000005F10071080130031D0030F0003008BD
:10012A00F00603199A28FF30B2003208F0000800DE
:10013A00003083122A06031DA4280A302906031D4B
:10014A00B0281A30FC00F830FD00FD0BAA28FC0B81
:10015A00AA2800000E2900302A06031DB6281430EA
:10016A002906031DC3283430FC00F130FD00FD0BC5
:10017A00BC28FC0BBC28000000000E2900302A060F
:10018A00031DC9282D302906031DD4287530FC000B
:10019A00E130FD00FD0BCF28FC0BCF280E290030E3
:1001AA002A06031DDA284B302906031DE528C33029
:1001BA00FC00CD30FD00FD0BE028FC0BE0280E29E9
:1001CA0000302A06031DEB285F302906031DF82894
:1001DA00F730FC00BF30FD00FD0BF128FC0BF128C5
:1001EA00000000000E2900302A06031DFE28913067
:1001FA002906031D0E290230FB007930FC009C30D1
:10020A00FD00FD0B0629FC0B0629FB0B0629000045
:04021A000E290800A1
:10021E0016208A110A128000840AA70A0319A80A56
:08022E00F003031D0F29080075
:100236008312A001A101A201A30152201C20AD013D
:100246002F2070088312AB007108AC0000307106D5
:10025600031D2F2900307006031D35290A30A90019
:100266000030AA002C08033C031D3B292B08843CC4
:10027600031840299130A900AA012C08003C031D4F
:1002860046292B08643C0318542901302C02031D0F
:100296004E292C302B02031854291430A9000030A3
:1002A600AA002C08013C031D5A292B082C3C0318D4
:1002B600682901302C02031D6229F4302B02031831
:1002C60068292D30A9000030AA002C08013C031D26
:1002D6006E292B08F43C03187C2902302C02031DDE
:1002E6007629BC302B0203187C294B30A90000303C
:1002F600AA002C08023C031D82292B08BC3C0318CB
:10030600902903302C02031D8A2984302B020318FE
:1003160090295F30A9000030AA000530AD000330F7
:10032600AE000530AF00B001652070080319B3298F
:1003360000302106031DA12900302006031DB12926
:10034600A201A3019D2085149D2005159D2005165B
:100356009D2085160130A0000030A100851D9B2937
:1003660000302306031DB92900302206031DC929C2
:10037600A001A1019D2085129D2005129D20051139
:100386009D2085100130A2000030A3009029CA29C3
:02400E00D400DC
:00000001FF
